:100000006400382185013F28DC2920344D344834F0
:100010007A342034003420342034203400345534F1
:100020005334423400344C3453344234003450346A
:10003000523447340034443446344D34203433345D
:100040002E343034203400342D34203456344B34A4
:100050003334423448345234003420342034203491
:100060004F34763465347234203400345234613481
:100070006E346734653420342034203400348601F3
:100080000A211B30BA202430BA202830C720322160
:1000900035219F019E110B118B168B179E12061A8C
:1000A0006F280530C720061A6F2841211E1E5E28C2
:1000B0002D30BA203630BA20352155281408970043
:1000C000150898001608990077211730BA203521B5
:1000D000061E55280530C720061E55289E16861F69
:1000E0007428061F7D288028061F7728792800306D
:1000F00081289E159F09033081289E15063081288E
:1001000009309E1A852892218628BF2141211E1E72
:100110008D282D30BA203630AD28861E9028AF208D
:1001200019089607031C9828950A031D9828940A15
:1001300018089507031C9D28940A17089407941F14
:10014000A328AF209F0977219E19A8280B30AD283E
:100150001F18AC280F30AD281330BA204828940956
:1001600095099609960A031DB928950A031DB92811
:10017000940A080089000908C320FF390319C6281A
:100180002421890ABB288200000000000800920098
:10019000CC20920BC8280034FF308F007E309000B6
:1001A00019309100910FD228900FD2288F0FD228AA
:1001B00000340F39860005150000051142308F000C
:1001C0008F0BE02800340A30900042308F008F0BF4
:1001D000E728900BE528003418308C009A019B0129
:1001E0009C019D011A30840004308E00333080075A
:1001F0008019F039801B0F398002840A8E0BF62893
:10020000960D950D940D9D0D9C0D9B0D9A0D8C0BCF
:10021000F2280800CC20851105110330D920CC200C
:100220000330D9200330D9200230D9200C302021CE
:10023000DE2006302021DE2001302021E3200034A2
:10024000851125290F39303E85159300130E29217C
:1002500013080F398600051500000511DE28C0308F
:100260002021DE2801302021E32802302021E3284C
:1002700083163730810010308500F03086008312FD
:1002800008001E12861106158614000086108101D2
:100290009401950196018615CC20CC20CC20CC2051
:1002A000861101089400051A5A2906110000061546
:1002B00096035329051E61290611000006159603B1
:1002C0005A2901088F0083160112000001168312BB
:1002D000950301080F06031963299503940C950CE7
:1002E000960C9413940C950C960C94130800EC2027
:1002F00030308D001A080F39031D81292030242148
:10030000822922211B0E22212E3024211B0822218A
:100310001C0E22211C0822211D0E22211D08222133
:100320000530BA2883128900093A0319A029BA2195
:100330009700890ABA219800890ABA219900080011
:100340000330922108308900BA219907031CAC2997
:10035000980A031DAC29970A8903BA219807031C40
:10036000B229970A8903BA219707970C980C990C20
:1003700097130800831608148312080808008316D0
:100380008B13831289001708CF21890A1808CF21FF
:10039000890A1908CF2183168B1783120800880059
:1003A0008316081555308900AA30890088148818EA
:1003B000D729081283120800A000030EA1000B1910
:1003C0001E160B11210E8300A00E200E0B1109002A
:02400E00F23F7F
:00000001FF
